:1000000000308A009C2D00000A108A100A11820715
:1000100028340C34013406340A108A100A1182077D
:10002000543465346D3470343A34203425343534E6
:100030002E3433346634B0344334203400340A1060
:100040008A100A11820754346C3461346B343A34A8
:100050002034253435342E34333466346B34503404
:100060006134003483168510831285106400A63035
:10007000F700F70B3928831685146400A630F700C3
:10008000F70B4028851483120034B7013708073C6A
:10009000031C6528831685108312851064000000F8
:1000A0000314B60C03185628851057288514831698
:1000B000851064001330F700F70B5C2800008514EE
:1000C000640000008312B70A46280034B6013608DF
:1000D000073C031C88288316851083128510640052
:1000E00000008316851464000230F700F70B7628B1
:1000F0008514831285187E2803107F280314B70CFB
:1001000064002730F700F70B83280000B60A672841
:100110003708F800003448308400831300080319BE
:10012000A2280130F800BF30F7006400F70B9528D3
:10013000F80B93284A30F700F70B9C280000640066
:10014000800B91280034AD013220CC30B600452020
:100150004430B6004520AD08031DB228662078085B
:10016000AD00AB283220CC30B6004520BE30B60002
:10017000452066207808AE0066207808AF002F087A
:10018000B1002E08B0003108B7003008B6008E303C
:10019000F7003708F8003608F900FA01B71FD5282C
:1001A000F809F909F90A0319F80AF808031DE22801
:1001B0007908F800F9010830F702F808031DE22871
:1001C000F701EB280310F81BE928F90DF80DF703E8
:1001D000E228B71FF8137708B6007808B700790847
:1001E000B8007A08B9003908BD003808BC003708E3
:1001F000BB003608BA00C101C001BF018330BE0098
:100200003A080319C529C6003E080319C529C602C4
:10021000031C0F297F30C6070318C5291529813013
:10022000C602031CC5290319C5294608F700F801B1
:10023000F901FA01C5013B08C400C4173C08C3001A
:100240003D08C2001930C6004108C202031838290F
:100250000130C30203183829C40203183829C50223
:1002600003183829C50AC40AC30A4108C2076A2903
:100270004008C302031853290130C402031853294C
:10028000C50203185329C50AC40A4008C307410818
:10029000C207031C6A29C30A031D6A29C40A031D75
:1002A0006A29C50A6A293F088038C40203186929E7
:1002B0000130C50203186929C50A3F088038C40700
:1002C0004008C307031C4729C40A031D4729C50A60
:1002D00047297A14C60B6D2978290310C20DC30D66
:1002E000C40DC50D0310FA0DF90DF80DC70D242925
:1002F000471C80290310F80CF90CFA0CC70C832951
:10030000F7030319C529C71BAC290310C20DC30D80
:10031000C40DC50D4108C202031898290130C3025B
:1003200003189829C40203189829C502031CBB2985
:100330004008C3020318A3290130C4020318A329EB
:10034000C502031CBB293F088038C4020318AC292E
:100350000130C502031CBB29FA0A031DBB29F90A97
:10036000031DBB29F80A031DBB29F70A0319C52978
:10037000F80CF90CFA0C3B08C6003F08C606C61F6D
:10038000C329F817C929F813C929F701F801F90198
:10039000FA017A08B5007908B4007808B300770844
:1003A000B200C830C8008B203208F7003308F800CC
:1003B0003408F9003508FA00EB2D8E30F7002E08CE
:1003C000F8002D08F900FA01F808031DF129790851
:1003D000F800F9010830F702F808031DF129F701C8
:1003E000F9290310F81BF829F90DF80DF703F12985
:1003F000F813072E4E18FE298611FF29861583163D
:1004000086118312CE18062A0611072A06158316AE
:10041000061183124E190E2A86100F2A861483168F
:1004200086108312CE19162A0610172A0614831670
:1004300006108312861783168613640083128613B0
:100440008316861383120034CC08031D292A8713D0
:100450002A2A8717A0132008831687008312CD0E3F
:100460004D08CE00FA21CD0E4D08CE00FA216400D1
:100470000C30F700F70B3A2A3D2A00341430C8003C
:100480008B208713A01320088316870083128613FE
:10049000831686138312AD012D08023C031C582AD3
:1004A0000230C8008B200330CE00FA21AD0A4C2A5E
:1004B00064000C30F700F70B5B2A5E2A0230CE0096
:1004C000FA2164000C30F700F70B642A672AAD01AB
:1004D0002D08023C031C782A2D080420AE00CC0114
:1004E0002E08CD0024220230C8008B20AD0A682AD5
:1004F000102E01304802CA004908023C031D822A1E
:100500004030CA074A088038CB00CC014B08CD00E8
:100510002422003447080C3A0319982A063A031992
:10052000A02A073A0319A62A053A0319AB2AB02ACA
:10053000CC010130CD0024220230C8008B20BC2A1F
:100540000130C8000230C9007922BC2A0130C8003D
:10055000C9007922BC2ACC011030CD002422BC2A4B
:1005600047081F3C031CB62A0730C7050130CC00E2
:100570004708CD002422BC2A0034470803192D2B3C
:10058000CF004B0803192D2BCF070318CE2A7F303D
:10059000CF02031C2D2B03192D2BD22A8130CF071C
:1005A00003182D2B4F08F700F801F901FA0148084C
:1005B000D300D3174908D2004A08D1001830CF0021
:1005C000D001511CFB2A4E08FA07031CED2AF90A38
:1005D000031DED2AF80A0319D0174D08F907031C6B
:1005E000F42AF80A0319D0174C08C900C91749089A
:1005F000F8070318D017D00DF80CF90CFA0CD30C2F
:10060000D20CD10C0310CF0BE02A0130F7070318EE
:100610002D2BF81B122BD30DFA0DF90DF80DF70346
:1006200003192D2BD31F232BFA0A031D232BF90AA1
:10063000031D232BF80A031D232BF80CF90CFA0CCD
:10064000F70A03192D2B4808D0004C08D006D01FFC
:100650002B2BF817312BF813312BF701F801F90187
:10066000FA010034F701F801F901FA01CF01D001D4
:10067000D101D2014E084D044C044B040319702BD8
:100680002030D3000310C70DC80DC90DCA0DCF0D02
:10069000D00DD10DD20D4E085202031D592B4D081D
:1006A0005102031D592B4C085002031D592B4B08B6
:1006B0004F02031C6A2B4B08CF024C08031C4C0F43
:1006C000D0024D08031C4D0FD1024E08031C4E0FE3
:1006D000D2020314F70DF80DF90DFA0DD30B422BCE
:1006E0004F308400831300340408BF003E08C1006B
:1006F0000319932B3D08CA003C08C9003B08C800F9
:100700003A08C700CE01CD012030CC008230CB00AA
:10071000BD227A08BD007908BC007808BB007708C4
:10072000BA00C10B7A2B3D08CA003C08C9003B083F
:10073000C8003A08C7004708B63CC700FA01480895
:10074000CB00C8170310C80CC90CCA0CFA0CF90C62
:10075000F80CF70CC70BA22BCB1FB92BF709F80924
:10076000F909FA09F70A0319F80A0319F90A03192A
:10077000FA0A7A08BD007908BC007808BB0077083F
:10078000BA00BD1FD02BBF03BF16BA09BB09BC09F5
:10079000BD09BA0A0319BB0A0319BC0A0319BD0A29
:1007A0003B30C6009A30C500CA30C400C3010A30CD
:1007B000C1003E080319BF0A3D08CA003C08C90031
:1007C0003B08C8003A08C7004608CE004508CD00DF
:1007D0004408CC004308CB0032230008BA00840A46
:1007E0000008BB00840A0008BC00840A0008BD00A1
:1007F000FD308407F708031D102C3E0A410203193F
:10080000102C3F080319122C0F39410203190A2C2E
:100810000318422CBF1B422C3F1B122C20303E2CB5
:100820002030BF05BF1E202CBF123E08031DBF0392
:100830007708BF002D30C7008A223F08F700BF01AC
:100840003E084102031D2E2C7708BF002E30C70042
:100850008A223F08F7002030BF0500303030BF1E2D
:100860003E2CBF123E08031DBF037708BF002D308A
:10087000C7008A223F08F700BF013030F70777082A
:10088000C7008A224608CA004508C9004408C800B3
:100890004308C700CE01CD01CC010A30CB00322382
:1008A0007A08C6007908C5007808C4007708C30034
:1008B000C10BDC2B003480308318BA06BF01C001A5
:1008C0003608BE003A08BE06350803194B2DBD0098
:1008D000F70039080319542DBD020319F02C031C2D
:1008E000AE2C3A08C300C3173B08C2003C08C10045
:1008F000C0010310C30CC20CC10CC00CBD0B782C82
:10090000BE1F852C3F14682D3F103D103F16383018
:10091000840083137D2D3F12BE1B982C3D1CA32CFD
:10092000C30CC20CC10CC00CF70A0319632DA32C15
:10093000C31BA62C0310C00DC10DC20DC30DF703C0
:100940000319632D982C3F17102D3F133608BE0056
:10095000BE1FAC2CC3175C2DC3135C2D3908BD0022
:10096000F7003508BD023608C300C3173708C200B8
:100970003808C100C0010310C30CC20CC10CC00C6C
:10098000BD0BBA2CBE1FC72CBF14682DBF103D1065
:10099000BF163C30840083137D2DBF12BE1BDA2CA2
:1009A0003D1CE52CC30CC20CC10CC00CF70A03198A
:1009B000632DE52CC31BE82C0310C00DC10DC20D27
:1009C000C30DF7030319632DDA2CBF17102DBF13C6
:1009D0003A08BE00BE1FEE2CC3175C2DC3135C2D5E
:1009E0003A08C300C3173B08C2003C08C100BE1F41
:1009F000FD2CC3133F15682D3F11C0013D10383049
:100A0000840083137D2DBE1B262D3608BE003D1CA1
:100A1000102DC30CC20CC10CC00CF70A0319632DB6
:100A2000C01F212DC10A031D212DC20A031D212D26
:100A3000C30A031D212DC30CC20CC10CF70A0319F4
:100A4000632D3F1BA52CBF1BE72C452D8030C30613
:100A5000C31F2E2D682D3A08BE003B2D3608BE0060
:100A6000C308031D3B2DC208031D3B2DC108031DF8
:100A70003B2DF7015C2DC31B452D0310C00DC10D8F
:100A8000C20DC30DF70B3B2D632DBE1F492DC317A0
:100A90005C2DC3135C2D3908F7003A08C3003B08EE
:100AA000C2003C08C1005C2D3508F7003608C300C1
:100AB0003708C2003808C1004308F8004208F900AE
:100AC0004108FA009B2DF701F801F901FA019B2D6D
:100AD000C001C109C209C309C009C00A031D762D9E
:100AE000C10A031D762DC20A0319C30A3F18842CBC
:100AF000BF18C62C3F19FC2C2B2D0008C107031C66
:100B0000872DC20A031D872DC30A03193D148403D0
:100B10000008C207031C8F2DC30A03193D14840368
:100B20000008801F803AC30703183D143F1A8B2C1E
:100B3000BF1ACD2C032D0034840183131F3083058D
:100B400083161F149F141F159F1107309C00FF3040
:100B50008312A00083161F109F141F159F151F13CB
:100B600083121F179F1783169F1783121F14831654
:100B7000091283129412A012200883168700831290
:100B800020162008831687008312A01120088316E0
:100B9000870001308312940000308316940001080E
:100BA000C73908388100831290010030F8009200A4
:100BB00000308316920007309C0005086400023064
:100BC000F700F70BE12DE42D1C0883120D1383169B
:100BD0009D018312A3287A08AC007908AB0078083D
:100BE000AA007708A900E330A8003830A7005E30DB
:100BF000A6007B30A5001F151F19FC2D1E08FA004A
:100C000083161E088312AD001E08AE00DD297A0887
:100C1000A4007908A3007808A2007708A1003E2A62
:100C20000130C800C9007922AD012D080C20AD0AA1
:100C3000F700C7008A2206302D02031D152E04304E
:100C400084002C08BD002B08BC002A08BB00290822
:100C5000BA000330BE007423B030C7008A2243308C
:100C6000C7008A222030C7008A220130C800023023
:100C7000C900792283142408B8002308B700220889
:100C8000B6002108B500BC01BB012430BA00843095
:100C9000B9005B247708AD007808AE007908AF0092
:100CA0007A08B000CA007908C9007808C800770837
:100CB000C7002808CE002708CD002608CC0025084C
:100CC000CB00BD227708B1007808B2007908B300E4
:100CD0007A08B40083107A08B8007908B700780859
:100CE000B6007708B500BC01BB017030BA00823095
:100CF000B9005B247708B5007808B6007908B7001A
:100D00007A08B800B90139081F20B90AF700C700EE
:100D10008A2206303902031D832E043084003808ED
:100D2000BD003708BC003608BB003508BA000330E8
:100D3000BE0074236B30C7008A225030C7008A225D
:100D40006130C7008A226430C8008B20EA2D63001E
:02400E0039393E
:00000001FF
